:020000005E2977
:080008008C0003088D00083094
:1000100081008E21E2200D0883008C0E0C0E0B1146
:100020000900AA00ED3E031837342A0882073F343E
:1000300006345B344F3466346D347D3407347F349A
:100040006F3477347C3439345E347934713400342D
:1000500040340834820700340A340B340C34013441
:10006000023403340D340434053406340E340734BA
:10007000083409340F348207553455345434543419
:10008000533453345334523452345234513451343F
:100090005034503450344934493449344834483465
:1000A000483447344734473446344634463445347C
:1000B000453445344534443444344434433443347F
:1000C0004334433442344234423442344134413480
:1000D0004134413440344034403440344034393485
:1000E00039343934393439343834383438343834AC
:1000F00038343734373437343734373436343634A9
:1001000036343634363435343534353435343534A4
:10011000353435343434343434343434343434349D
:100120003434333433343334333433343334333496
:10013000323432343234323432343234323432348F
:100140003134313431343134313431343134313487
:10015000313430343034303430343034303430347E
:10016000303430343034303429342934293429348B
:100170002934293429342934293429342934283498
:10018000283428342834283428342834283428348F
:100190002834283427342734273427342734273485
:1001A0002734273427342734273427342634263479
:1001B000263426342634263426342634263426346F
:1001C000263426341D0882074C29A929F528E82958
:1001D0000D2AB929B929142A4C294C294C294C2912
:1001E0004C294C294C294C294C29190803398207E0
:1001F0003A293A29FC280800AB0A0A302B02031DD1
:100200003929AB01900A0A301002031D39299001E7
:10021000910A11120A301102031D39299101920A23
:1002200012120A301202031D39299201930A131285
:100230000A301302031D39299301940A14120A305B
:100240001402031D39299401950A15120A3015026A
:10025000031D39299501960A16120A301602031D4C
:1002600039299601970A17120A301702031D3929F6
:1002700097010800A217AB01900191019201103083
:100280004629103090009014910092009300940041
:100290009500960097000800190A9D000800A90122
:1002A0000A30A802031C5629A90A5129A8072808C0
:1002B000CF002908A8004F08A90008008B0183017E
:1002C0008316D1308100F83085000030860083121B
:1002D00085010514860198170F309D0099009A0139
:1002E0009B019C019F01A001A101A201A301A40106
:1002F000A501A601A7014121083081008B168B17AB
:100300008029050818399B00183C03198D291C14F5
:100310001B081804F83E2A20990008008601980A54
:1003200008301802031C9C299C101C189C141C10DB
:100330009801851485109E2905100514812118083F
:10034000840004160008112084160412000486009C
:1003500008009808031D0B281908860005150511CB
:100360000F3911208600190E0F3991009901990952
:100370000800AB0F0800980105150610AB0FBE2949
:10038000061405118316FF3086008312A801061893
:10039000CB29A80AC729831686018312191CD629DE
:1003A0005F3028023B209E00A117ED29A1134F21A9
:1003B000290890004F21280892000319E2292908F2
:1003C000910008001216290891000319111608005F
:1003D000980803190322191CFB290F301E059000F1
:1003E0001E0E0F399100103092009300940095007A
:1003F0009600970008001808840004161E080139AA
:1004000080009E0C08008316FF30860083120608C9
:100410009E00831686018312080085148510051539
:10042000860A00000000102A98080319182A0800FC
:100430009C191D2A99019C151C159908031D222A37
:10044000412190019C181C19262A02211C159C1C74
:100450001C1103221E089F049F060830AA009F0D4E
:10046000031C332A0221AA0B2F2A1E089F00080012
:02400E00FA3F77
:00000001FF
